:100000009128A0003F200C080D0403198C2886209D
:1000100084132008800664000D280E288C0A03191A
:100020008D0F0B2880068C288F0022088400200961
:10003000402084138F0803198C28F03091000E089B
:1000400080389000F03091030319910003198F0359
:1000500003198C282B28552003010C1820088E1F0B
:1000600020088E0803190301900F382880061F28E6
:100070003928000022284320FF3A80054028FF3A13
:10008000841780058C28940006309419053084006C
:1000900000308A001408073982070134023404341E
:1000A000083410342034403480340D080C04031913
:1000B0008C0A80300C1A8D060C198D068C188D0652
:1000C0000D0D8C0D8D0D8C288F018E00FF308E074D
:1000D000031C8F07031C8C2803308D00DF30722037
:1000E00066288D01E83E8C008D09FC30031C7B28BE
:1000F0008C07031878288C0764008D0F78280C185B
:1001000081288C1C85280000852808008C098D0911
:100110008C0A03198D0A08008313031383126400E9
:1001200008008316850103308600831205118316AB
:100130000511831285118316851183122C083B202B
:100140002D083B202E083B202F083B2030083B2069
:1001500031083B20B6012830AA001930B400013024
:10016000B3006400063033020318CE280515831649
:100170000511831285118316851183128721323070
:1001800064200511831605118312851583168511C8
:100190008312872132306420B30FB1288511831672
:1001A000851183126400061CF32832306420640039
:1001B000061CDC28D728F3280530A2001030A00048
:1001C00078308E00043014205A308E000230142013
:1001D00064308E00023014206E308E000430142003
:1001E00032306420B3299C2164002B08013C031D9C
:1001F0001A29051583160511831285158316851195
:1002000005308312A2001030A00064308E0004304C
:1002100014205A308E0002301420B430AC00E82193
:100220007830AC00E821B60A6400361C19293F2159
:100230001A2963210511831605118312851183166E
:10024000851183122421D2289D30AC00D230AD001C
:100250008F30AE006430AF009D30B000D230B100BE
:10026000E8218F30AC006430AD009D30AE00D2305C
:10027000AF008F30B0006430B100E82108000130D9
:10028000B300640004303302031862299630AC00D6
:10029000D230AD009630AE006430AF009630B00082
:1002A000D230B100E821BE30AC006430AD00BE30C9
:1002B000AE00D230AF00BE30B0006430B100E821F3
:1002C000B30F412908000130B30064000430330249
:1002D000031886299630AC00D230AD009630AE00BF
:1002E0006430AF009630B000D230B100E821643005
:1002F000AC006430AD006430AE00D230AF0064308A
:10030000B0006430B100E821B30F6529080024086B
:100310008C0025088D0055200C08A4000D08A500B0
:100320005F302405A6000530A2001030A00026088A
:100330008E00043014200800A701AB010130B20088
:10034000640032082A02031CAB2964008618A9291C
:10035000A70AB20FA029640034082702031CB2299F
:100360000130AB00080064008618BE29051583160D
:1003700005118312851583168511831205118316C5
:100380000511831285118316851164008312061CE2
:10039000E729323064206400061CD029CB29E729E4
:1003A0000530A2001030A00078308E0004301420F8
:1003B0005A308E000230142064308E000230142037
:1003C0006E308E000430142032306420D228B329DD
:1003D0000130B50064001530350203181D2A2C08C1
:1003E0008C008D0106308400043001202D088C0023
:1003F0008D0106308400083001202E088C008D010C
:1004000006308400803001202F088C008D010630DA
:1004100084004030012030088C008D0106308400BB
:100420002030012031088C008D010630840010300E
:0C04300001200C306420B50FEA29080000
:02400E00F53F7C
:00000001FF
